:100000000EC01BC01AC019C018C017C016C015C03A
:1000100015C013C012C011C010C00FC00EC01124F3
:100020001FBECFEDCDBF10E0A0E6B0E001C01D9235
:10003000A236B107E1F720D088C0E2CF1F920F921D
:100040000FB60F9211248F939F9395B19F3F11F498
:10005000C39A8895389B05C082EA87B9909360005F
:1000600004C081EA87B9909361009F918F910F90AE
:100070000FBE0F901F90189580E285BF86E080BD6F
:10008000789481E288BB8BE287BB87E087BD9FEFD6
:100090009DBD81E680BF81EA87B996B982EA87B9BA
:1000A00040E050E0E0E0F0E08895889560916000E5
:1000B00080916100653B80F4882311F09FEF01C0BF
:1000C00091E04115510521F04150504009F4C09A8A
:1000D000C59AE3E6F9E011C090E070E024D08659BB
:1000E000914310F09FEF01C091E0C098309719F054
:1000F000319709F4C5984FE855E28EB5292F33277B
:1001000027FD3095280F311D8FEF2F3F380719F449
:1001100020E030E006C081E02030380711F42FEFF6
:1001200030E02EBDC1CF5527002480FF02C0060E4F
:10013000571F660F771F6115710521F096958795FA
:0E014000009799F7952F802D0895F894FFCF22
:02000004008278
:03000000C154FFE9
:00000001FF
